:020000040800F2
:10000000001800200508000835050008390500081B
:1000100000000000000000000000000000000000E0
:10002000000000000000000000000000350500088E
:10003000000000000000000035050008350500083C
:1000400035050008350500083505000835050008A8
:100050003505000835050008350500083505000898
:100060003505000835050008350500083505000888
:100070003505000835050008350500083505000878
:100080003505000835050008350500083505000868
:100090003505000835050008350500083505000858
:1000A0003505000835050008350500083505000848
:1000B00035050008350500083505000899010008D8
:1000C000284B10B51A88284B12041B881A43274B5B
:1000D000198849084900885A254908801988023139
:1000E00089B21980198849084900885A214908802D
:1000F0001988023189B21980198849084900885A3B
:100100001D49088019881D48023189B21980198853
:1001100049084900895A1A4A11801A881949023235
:1001200092B21A801C880288944213D902881C88D3
:100130000832121B92B20A80028892B21A801249C7
:10014000124B0A881343124A1A40302353409BB281
:100150000B8010BD0F4804881A889442E6D3082308
:100160000B80ECE70C6000400A6000400460004037
:100170004C6000404E600040506000400260004013
:10018000526000401A600040005C00408080FFFF29
:10019000BF8FFFFF006000409449F8B50B88944C76
:1001A000002B3AD00A88934B9A4234D1002302257F
:1001B000914A924F1380924A1380924A1380924A36
:1001C0001380924A1380924AD08FA843D087D08F51
:1001D000013DA843D0878F481735FB8705808E489F
:1001E000343505808D480835058080258C486D01A3
:1001F000058080258B4805808020FB878A4B000680
:1002000023808A4B18608023D08FDB000343D38781
:10021000874B884A1A8000230B8023881BB2002B4F
:1002200000DBC4E02388844A774F134080221343C5
:10023000238023881B0500D49CE0804D7F232A78EF
:1002400011009943714B1980E9886B4B198000218B
:100250006C4B19803B88FF318B4313433B806023F9
:100260001A4208D08022764B12051B8828009B1862
:100270009847634B188060232A78134052B2002AB3
:100280004DDA002B14D16A78062A0FD16A88110A38
:1002900002291AD003291BD0012920D1694B12262B
:1002A000694A99B21180694A1B0C1380544B1E8015
:1002B0002288674B1343674A1A40C0239B0153406F
:1002C0009BB22380FFF7FCFE47E05E4B1233E6E76C
:1002D000D2B2012A0FD0002A03D0022A15D01E0064
:1002E000E4E7584B584A243399B21180574A1B0C03
:1002F00013800426DAE7534B534A283399B211800E
:10030000524A1B0C1380544ED0E74E4B4E4A7C335E
:1003100099B211804D4A1B0C1380504EC6E7002B3A
:1003200009D16B78052B06D13A886B88D2B21B02B3
:1003300013439BB23B8000212388494A1340494A1A
:1003400013439BB22380484B198023881A43474BA1
:100350001A40474B5A4092B22280284BDB8F5B05F4
:1003600007D580222F4B1A800023244AD3872E4B97
:100370002380F8BD60213B880B40402BEDD13B88AA
:100380001342EAD1264A3B4B2C481B881188802215
:1003900012059B18C9B298472288324B13432D4A45
:1003A0001A40C0239B0153409BB22380D5E7802293
:1003B00023881342D1D023882F490B408021090282
:1003C0000B432380114B1B88934200D17AE7FF2017
:1003D0000D4B19888143C0D01988090A0A43114975
:1003E0000A801A8802401A80B7E7C0460E600040B3
:1003F000005C00403CA5000000600040065C00403E
:100400000260004004600040066000400860004058
:10041000025C0040505C0040186000401C600040DE
:100420001E6000404C5C00402032000000E100E013
:10043000585C00400080FFFF8F0F000054600040B8
:10044000106000407C0400080A6000400C6000401E
:100450008081FFFF8FBFFFFF2A0300001E03000003
:100460008F8EFFFF8080FFFF1A600040BFBFFFFF3D
:1004700030300000126000400F8FFFFF12010002B9
:10048000FF000008C016DC0503020102000109029A
:100490001200010100803209040000000000000089
:1004A000040309042A0349006E00660069006E0017
:1004B0006900740065004E00650073004C0069001F
:1004C0007600650073002E0063006F006D00000071
:1004D000000000000000000000000000000000001C
:1004E000000000000000000000000000000000000C
:1004F00000000000000000001E0349004E004C00F8
:10050000200052006500740072006F002D00500042
:1005100072006F0067000000000000000000000093
:1005200000000000000000000000000000000000CB
:1005300000000000FEE7FFFF004801E02301ADDE00
:10054000FEE7C04602B4714649084900095C49000B
:100550008E4402BC7047C046411D000000616561C9
:1005600062690001130000000536532D4D00060C92
:10057000074D09011901FFFF03B471464908400006
:100580004900095A49008E4403BC7047411D0000D0
:100590000061656162690001130000000536532D9A
:1005A0004D00060C074D09011901FFFF70470A4B6A
:1005B0000A4A10B55A600A4A5A600122DC6814429D
:1005C000FCD11A6101220180D9681142FCD120229C
:1005D000DA6060321A6110BD0020024023016745D5
:1005E000AB89EFCDFF2370B53F4D2B804378C68894
:1005F000102B00D075E0C478818880783B4B01389F
:100600005A69082800D968E0FFF79CFF0567672B47
:100610003D314B5363008A1E8E241D2A19D8344A5B
:100620005A60344A5A600122D8681042FCD1022232
:100630001A618022890212058918422259611A61C1
:10064000C046413ADC681440FCD12022DA606032B6
:100650001A612C70284BAAB22D0CF0B25A819D81E0
:1006600070BD60001018FFF7A2FF0024F1E7002C16
:1006700035D10BB2002B32DB80231B05C8181F4974
:10068000FFF795FFE5E704226A705A69AA705A6974
:10069000120AEA705A69120C2A715B691B0E6B719F
:1006A000E3E702236B701388AB7013881B0AEB70AF
:1006B000DBE7002C13D10BB2002B10DB80231B05D2
:1006C000C91802236B700B88AB700B881B0AEB7088
:1006D000BFE70B4B0B4ADA60C7E78B24B9E78E24E0
:1006E000B7E780232B70B5E7EC060020002002401E
:1006F00023016745AB89EFCD00600040FFFF00009C
:1007000000ED00E00400FA05FFFFFFFFFFFFFFFF21
:10071000FFFFFFFFFFFFFFFFFFFFFFFFFFFFFFFFE9
:10072000FFFFFFFFFFFFFFFFFFFFFFFFFFFFFFFFD9
:10073000FFFFFFFFFFFFFFFFFFFFFFFFFFFFFFFFC9
:10074000FFFFFFFFFFFFFFFFFFFFFFFFFFFFFFFFB9
:10075000FFFFFFFFFFFFFFFFFFFFFFFFFFFFFFFFA9
:10076000FFFFFFFFFFFFFFFFFFFFFFFFFFFFFFFF99
:10077000164B174A9BB21382164B9BB253826846A4
:100780001C300F4A0F4B0430043001681140C91A65
:10079000FAD1094A094B043801681140C91AF2D14B
:1007A0007B460A3303600438013303600CE00A4BD4
:1007B0000A4A1A60FBE7C0460000FFFF000000087D
:1007C000FFFFFF0F0000000100207047E505000853
:1007D00000600040AD05000800300040AAAA0000FB
:1007E000FFFFFFFFFFFFFFFFFFFFFFFFFFFFFFFF19
:1007F000FFFFFFFFFFFFFFFFFFFFFFFFFFFFFFFF09
:10080000FFFFFFFF09490A4A0A4B9B1A03DD043B1D
:10081000C858D050FBDC0849084A0020521A02DDB3
:10082000043A8850FCDC02F02BFA00005049000822
:1008300000000020300400203004002008070020C1
:1008400070B50E4B1A68537A55685C18E4B2A3422F
:100850000ED1537A0A48CB1853720378591AC9B289
:1008600001700020814202D198230130D37070BD05
:1008700006780130EE540133DBB2E8E79004002043
:1008800095040020FF23F7B5C34C0500238083792E
:100890000093407801380A2801D901F0A3F9FFF745
:1008A0006BFE0B00B404CC05A1094B08A1098E090D
:1008B0001C07A407EE074808A878AB8819281BD89E
:1008C000FFF75AFE1E002600EC00B8016002D202BB
:1008D0004E03D603E703F203F903000408041004EF
:1008E00038044704550464048B048B048B041A00F9
:1008F0001A001A004A0255028C23237000F007FEEA
:10090000E023A64A1B0351690B4353610023F4E71C
:10091000152B01D900F064FC1800FFF72DFE16001E
:1009200021002E003B00480055005F006C0076005F
:1009300081008D009A006104610461046104610416
:100940006104A70061046104B40090234022DB0528
:10095000196891431960D9680A43DA600023CCE72B
:100960009023DB051A688E490A401A608022D968F4
:1009700052000A43DA600023BFE79023DB051A68C0
:1009800088490A401A608022D968D2000A43DA6096
:100990000023B2E79023DB051A6883490A401A60F6
:1009A0008022D96852010A43DA600023A5E7902328
:1009B000DB051A687D490A401A608022D968D20195
:1009C0000A43DA60002398E70122794B19689143C2
:1009D0001960D9680A43DA6000238EE79023DB05AB
:1009E0001A6874490A401A608022D96852030A437F
:1009F000DA60002381E704226D4B19689143196086
:100A0000D9680A43DA60002377E790230122DB05E7
:100A1000196891431960D9680A43DA6000236CE7CA
:100A2000654B66491A680A401A608022D968D20468
:100A30000A43DA60002360E79023DB051A68604907
:100A40000A401A608022D968D2050A43DA6000237E
:100A500053E79023DB051A6858490A401A60802240
:100A6000D968D2040A43DA60002346E79023DB0505
:100A70001A6854490A401A608022D96852050A430C
:100A8000DA60002339E790230122DB0519689143DE
:100A90001960D9680A43DA6000232EE7152B00D9C4
:100AA000A1E31800FFF768FD160021002C003700B5
:100AB00042004D00570062006C0090009A00A500B3
:100AC0009F039F039F039F039F039F03B0009F0308
:100AD0009F03BB0090234021DB051A688A431A60FC
:100AE000DA688A43DA60002307E79023DB05196898
:100AF0002B4801401960DA680240DA600023FCE606
:100B00009023DB051968274801401960DA68024024
:100B1000DA600023F1E69023DB05196822480140E2
:100B20001960DA680240DA600023E6E69023DB050C
:100B300019681E4801401960DA680240DA60002333
:100B4000DBE601211A4B1A688A431A60DA688A4385
:100B5000DA600023D1E69023DB05196815480140CF
:100B60001960DA680240DA600023C6E60421104BFF
:100B70001A688A431A60DA688A43DA600023BCE69E
:100B800090230121DB051A688A431A60DA688A43D8
:100B9000DA600023B1E6C046F406002000100240EF
:100BA000FFFEFFFFFFFBFFFFFFEFFFFFFFBFFFFFAA
:100BB00000040048FFFFEFFF00080048FFFFFFFBB5
:100BC000FFFFFFBFFFFFFFEFC14BC24819680140A5
:100BD0001960DA680240DA6000238EE69023DB05B4
:100BE0001968BD4801401960DA680240DA600023E4
:100BF00083E69023DB051968B64801401960DA687E
:100C00000240DA60002378E69023DB051968B348D8
:100C100001401960DA680240DA6000236DE6902333
:100C20000121DB051A688A431A60DA688A43DA60B0
:100C3000002362E6152B00D9D8E21800FFF79CFCD0
:100C400016001E0027003000390042004900520003
:100C50005900610069007200D602D602D602D6029F
:100C6000D602D6027B00D602D60284009022402310
:100C7000D20511680B43136000233EE690228023C7
:100C8000D20511685B000B431360002335E6902208
:100C90008023D2051168DB000B43136000232CE690
:100CA00090228023D20511685B010B43136000235F
:100CB00023E690228023D2051168DB010B431360E9
:100CC00000231AE60123864A11680B4313600023B0
:100CD00013E690228023D20511685B030B43136057
:100CE00000230AE604237E4A11680B4313600023A5
:100CF00003E690220123D20511680B431360002301
:100D0000FBE58023724ADB0411680B431360002368
:100D1000F3E590228023D2051168DB050B431360B5
:100D20000023EAE590228023D2051168DB040B43FF
:100D300013600023E1E590228023D20511685B0552
:100D40000B4313600023D8E590220123D2051168DC
:100D50000B4313600023D0E5082B00D049E290221A
:100D6000D2055168073B0B4353600023C5E5082BB0
:100D700000D041E290220121D20553688B43536099
:100D80000023BAE5152B00D939E21800FFF7F4FB70
:100D900016001C00220028002E00340039004000FC
:100DA00045004B0051005800370237023702370226
:100DB000370237025F0037023702660090230822AD
:100DC000DB059A62002398E590231022DB059A62E6
:100DD000002392E590232022DB059A6200238CE514
:100DE00090234022DB059A62002386E5902380222F
:100DF000DB059A62002380E50122394B9A620023C9
:100E00007BE590238022DB05D2009A62002374E503
:100E10000222334B9A6200236FE590230122DB0507
:100E20009A62002369E58022294B92019A6200238D
:100E300063E590238022DB0512029A6200235CE5C1
:100E400090238022DB0592019A62002355E59023CE
:100E50008022DB05D2019A6200234EE59023012215
:100E6000DB059A62002348E5152B00D9CAE118007A
:100E7000FFF782FB16001C002200280038003E000D
:100E800043004A004F0055005B006200C801C801E2
:100E9000C801C801C801C8016900C801C8017000C3
:100EA00090230822DB059A61002326E59023102277
:100EB000DB059A61002320E590232022DB059A615F
:100EC00000231AE590234022DB059A61002314E5F4
:100ED00000080048FFFFFFFBFFFFFFBFFFFFFFEF22
:100EE0000004004890238022DB059A61002304E57A
:100EF0000122CC4B9A610023FFE490238022DB0582
:100F0000D2009A610023F8E40222C64B9A610023C2
:100F1000F3E490230122DB059A610023EDE48022B3
:100F2000C14B92019A610023E7E490238022DB0504
:100F300012029A610023E0E490238022DB059201F3
:100F40009A610023D9E490238022DB05D2019A61C3
:100F50000023D2E490230122DB059A610023CCE434
:100F600002226270152B00D97EE01800FFF7EAFA22
:100F70000B131B232B333A434A525A627C7C7C7CF2
:100F80007C7C6B7C7C7490230822DB051B691340FE
:100F900063800023B1E490231022DB051B6913401A
:100FA00063800023A9E490232022DB051B69134002
:100FB00063800023A1E490234022DB051B691340DA
:100FC0006380002399E490238022DB051B69134092
:100FD0006380002391E40122924B1B6913406380DC
:100FE00000238AE490238022DB051B69D200134092
:100FF0006380002381E402228A4B1B6913406380D3
:1010000000237AE490230122DB051B6913406380EF
:10101000002372E48022844B92011B691340638099
:1010200000236AE49023DB051B69DB0BDB03638091
:10103000002362E490238022DB051B6992011340A8
:101040006380002359E490238022DB051B69D201D1
:1010500013406380002350E490230122DB051B69C9
:1010600013406380002348E4002363708D3344E41D
:1010700080236E4ADB0251690B435361694B6C4913
:101080001A680A401A60D9686A4A0A43DA6000237B
:1010900033E4644B66491A680A401A60D968654AA5
:1010A0000A43DA60002328E45E4A614913680B4072
:1010B0001360002321E45B4A5E4B11680B4313600D
:1010C00000231AE457491B024A69D2B213434B6109
:1010D000002312E4534B1B691B0AA37001236370A6
:1010E00000230AE48023514ADB02516950480B4334
:1010F00053614C4B196801401960D8684D49014350
:10110000D960C0215069C9020143516104221968A4
:101110000A431A60022290219A62A022C905086837
:10112000D20202430A601968434A0A431A60002344
:10113000FFF7E3FB9022A023D205D168DB020B432B
:10114000D360384A3C4BD1680B43D3600023FFF790
:10115000D4FB9022D205136838490B401360314A02
:10116000374913680B4013600023FFF7C6FB90223A
:10117000A023D2051168DB020B431360294A2E4BD2
:1011800011680B4313600023FFF7B7FB9020C005E5
:1011900042692C499D000A40C021890029400A4328
:1011A0004261204A284851691B0A0140FF2005403E
:1011B0002943516115681F491B0229431160516978
:1011C00008400343536102239361936213681849F3
:1011D0000B4013600023FFF790FB0023FFF78DFB0C
:1011E0008D23FFF78AFB8D23FFF787FB8D23FFF706
:1011F00084FB8D23FFF781FB8D23FFF77EFB8D237F
:10120000FFF77BFB8D23FFF778FBAA88AD78032DD2
:1012100000D1D7E01AD8002D67D0012D69D09623D0
:10122000DFE0C0460004004800080048001002400B
:10123000FFFFAAAA0000555550550000FFFFFAFF16
:10124000AFAAFFFFFFFC000003FF0000042D00D148
:10125000E6E0802DE3D190230122DB0562709A62E3
:10126000196811431960C046186919681040914304
:101270001960D9689143D960F021002832D11968EA
:1012800091431960D9681143D9601F691E69C0462E
:101290001D69C046C0461C69C046C046C0461969A3
:1012A0008C46C046C046C046C046196901911968BF
:1012B00091431960D9689143D9600100174211D157
:1012C000110016420ED1023115420BD103311442E6
:1012D00008D163460431134204D1019BD631DB07A8
:1012E00000D5D139C04B997001E001F05FFA0023BD
:1012F00077E001F05BFA90228023D20511685B0051
:101300000B43136010239361116830330B43136058
:101310000823936280231168DB000B4313602023B2
:10132000936180231168DB010B4313608023936179
:10133000AE4BAF481968AF4C294319609D618025B9
:101340004169ED0229434161196821401960DE6855
:10135000A9490E43DE601E6826401E60DE680E430B
:10136000DE604669354345611D6825401D60DD68C6
:101370000D43DD60C0254669ED023543456104201B
:101380001D68284318600220A02598621668ED02A7
:10139000354315601E68994D35431D605569984E5B
:1013A000354055615A69974D2A405A611A68114370
:1013B00019605A69D2B25A61986198621A681440E9
:1013C0001C6094E7D2B2022A0ED00023032A08D070
:1013D0009733012A05D100238B4A8C4913708C4A1C
:1013E0001160814CFFF789FAE023814A1B035169A0
:1013F0000B43536190230122DB0519689143196067
:10140000D9681143D9605968114359609A611968C4
:101410000A4308211A607C4A11707D4A136066E70E
:10142000D2B29823012ADCD1E023714A1B0351690F
:101430000B43536101F03EF959E7E978A888AD788C
:101440000D2D00D1C3E029D8062D00D166E011D8BA
:10145000022D00D169E005D8002D54D0012D61D0B6
:10146000A02552E0042D00D19FE0052DF8D100F019
:10147000C7FC55E0092D00D1A0E007D8072D00D109
:10148000ABE0082DECD100F0CBFD49E00B2D00D1F5
:10149000A0E000D895E000F05BFE41E0222D47D0AF
:1014A00015D8102D00D19BE007D80E2D00D18BE070
:1014B0000F2DD5D101F0DCFA32E0202D00D177E0FC
:1014C00000D978E0112DCBD100F084FE28E0822DE8
:1014D00000D1EFE00AD8802D00D1A1E0812DBFD14D
:1014E0000123637000F0EEFEA07019E0852D00D19D
:1014F000E5E0862D00D1E8E0842DB1D101236370B1
:1015000000F0C4FCF0E700F0B5FF374C2570414B0C
:10151000A2B2240C5A8100989C81FEBD00F068FFA5
:101520000025F2E700F0F2FCFAE700F0BDFDF7E776
:101530009022D2055369324D84002B40C025AD0066
:1015400025402B435361294B2E4E5D6909023540DE
:10155000FF26344025435D611D68274C25431D60EF
:101560005F69050A37402D023D435D6102259D619B
:101570009D621F681F4D00B22F401F602027976299
:101580001F683C431C605C6934402143596100285A
:1015900001DA10219162C046C046102191614918BC
:1015A00091611A6815401D60BAE701F04FFAB7E77C
:1015B000194B1870B4E7194B1880B1E700F0D2FF4F
:1015C000AEE700F04FFDABE701F082FAA8E700F0CC
:1015D00097FFA5E700F038FEA2E700F0E1FE9FE7E5
:1015E00000F0B4FE9CE7C046F4060020000400486A
:1015F00000100240FFFFAAAA0000555550550000F8
:10160000FFFC000003FF0000000700200008004866
:10161000FC06002000600040880400203604002002
:10162000012190226170D205136808248B43136056
:10163000D36810258B43D360202394629561936116
:101640005369C34986000B40C021890031400B43D8
:101650005361C04BC0495F693940FF273E400E438C
:101660005E611E68BD4931431960010AA1405E698F
:1016700037400F4302215F61996199621968B84E42
:1016800031401960C046C04600B29461002800DABB
:101690009562C046C046C046C046C046C04690227D
:1016A0000821D2051B69916249189161AD4A1B0A54
:1016B000937035E70123637000F070FC14E7012399
:1016C0006370A94B1B78A3702AE702236370A74BB2
:1016D0001B88A3701B0AE37022E7EA78A988AD781B
:1016E000112D7BD007D8012D4ED0002D0DD0022D0D
:1016F0005CD0822646E0212D66D0222D6AD0122DA4
:10170000F7D10223102063706BE00127984B042669
:101710001B7810209F40FA43964B01921D68AF62E0
:101720006B6813406B6000F060FBAF616B683B431C
:101730006B60FA20400000F058FBFA20AF626B6843
:10174000019A400013406B6000F04FFBAF616B6883
:10175000013E3B43B6B26B60002EEAD10436FA205C
:1017600000F043FBAF626B68019AFA2013406B6094
:1017700000F03BFBAF616B68013E3B43B6B26B6070
:10178000002EECD12670C2E6794A7A4B12781E6898
:101790009540B56273681020AB43736000F025FB81
:1017A000B56173682B4373600026EBE70123704A31
:1017B00063701278704993406E4A9BB212680020A1
:1017C00001F076FFA070EFE701230020637001F0C5
:1017D000A7F9F7E7012310206370F8E70223002040
:1017E000637001F0F7F96080DEE7AB78AA88042B1C
:1017F0001DD007D8022B1FD024D8012B12D087234D
:10180000FFF77BF8072B26D003D8052BF7D15B4BCE
:1018100016E0082B24D0802BF1D100F04BFF0023E1
:10182000FFF76BF8564A1278A2706370F7E7554BD2
:101830001B78A3700123F8E7514B1A708322514B98
:101840001A70ECE74E4B4F4D1A7083232B7000F04B
:1018500051FF2B78EDE74C4B1A70120A5A70DEE7F5
:10186000494B1A78A2705A78E2709A782271DA7825
:1018700062711A79A2715B79E3710623D5E7A878C2
:10188000E9780238AA888A23092801D9FFF735F8B0
:10189000FEF758FE050A10151C232F3B40483B4B12
:1018A0001A800023FFF729F8384B1B881B041343C9
:1018B0009847F6E7FEF75CFF0300FFF71EF8344891
:1018C000036899B213040B430360EAE730490B68DD
:1018D0001B0C1B0413430B60E3E7042363702C4BC6
:1018E0001B681A0AA370E2701A0C1B0E2271637136
:1018F000D7E7022363705300254A1168CB181A8872
:10190000A2701B881B0AE370CBE7214B49001B68C0
:10191000CA52C6E71E4953000A68D31802220B6058
:101920006270ECE71A4B49001868411819600A8088
:10193000B7E78823FEF7E1FFAA781300303B2F2B8F
:101940003CD8E878032836D8FEF7FCFD383A243333
:10195000FFFC00000004004803FF00000000555594
:10196000FFFFAAAAF4060020880400203604002005
:1019700000070020FC06002004000200D90400201B
:10198000B8040020DA040020B90400203404002048
:1019900030040020A34B512A00D17AE027D8312A05
:1019A00055D00FD8002A35D0302A49D0B423FEF7BD
:1019B000A4FF9D4BEFE7B523FEF79FFF9B4BEAE7A4
:1019C0009B4BE8E7332A50D048D3502AEED1C022AF
:1019D000D20022801A7AA270DA78E2705A7A2271E2
:1019E0009A7A62719A78A2715B7CE3718FE57F2AA3
:1019F00000D982E0702A5BD2602A3BD0612A41D0B4
:101A0000522AD3D180221B889200A3701B0A228005
:101A1000E3707CE5FF21874BD1540132102AFBD1C2
:101A20000123824A5B425380814A53807D4A53801E
:101A30007D4A53800122804B1A700023FEF75DFF20
:101A4000AA88110AD9721A730023FEF756FFAA88D2
:101A5000110A59739A730023FEF74FFFAA88110ADF
:101A6000D9731A740023FEF748FFAA885A7400231A
:101A7000FEF743FF80235B002380AB886D4AD35C75
:101A8000A37044E580235B0023806C4B1B68DB78EC
:101A9000F6E7C022D2002280DA7AA2701A7BE270C6
:101AA0005A7B22719A7B6271DA7BA2711B7C9CE764
:101AB0005E4B28785C68614B1B68D9787F2800D919
:101AC00093E05F48009E067000290FD00020009030
:101AD000982900D18FE004E000200090D02900D1A7
:101AE00089E0554910300870FF2104E055490B602A
:101AF0009021D9706F3100917DE0072010400328BC
:101B000017D8FEF71FFD191B0214464B802A00D27E
:101B1000FDE4872A14D97032D2B2072A00D9F6E43C
:101B200000222270EA789A72AA881A80EFE43E4B6B
:101B3000ECE7B523FEF7E1FE3C4BE7E73C4BE5E77E
:101B4000A888E978C6B28D19BE22102D2CDC04328B
:101B5000002929D0DD78033AFF2D25D19D78013267
:101B6000FF2D21D10022D7B2B9421FD8364D002215
:101B7000AC464F01013F1F727701000A674498701D
:101B8000DA705A729A721A80DA721A735A739A73E6
:101B9000DA731A745A745F60264B9D19A854013287
:101BA000D3B29942FAD800222270B0E40132B718B9
:101BB000204D013FEF5DFF2FD5D0C122F4E7AB7878
:101BC000002B04D0402B07D0D223FEF796FE2370C3
:101BD000AA88194B1A709AE480235B002380164B65
:101BE0001B784DE78023FEF788FED82900D073E7E5
:101BF00080215C68D97000215972DB78902B00D06D
:101C000085E4712A00D082E40E4BAA881B685968CB
:101C10000A70AA885968120A4A705A7A02325A72AD
:101C200075E4C046600400207404002038040020DD
:101C30004C040020DB040020980400208C040020C9
:101C40009504002090040020EC040020F0B585B03D
:101C500001932A4B00901C6829482043186058695A
:101C60000C02C0B220435861022098619862186843
:101C7000244C49B22040902418600820E405A0615B
:101C8000002901DA1021A16265691F499000C0276F
:101C90008C460D400100BF0039400D436561FF24B3
:101CA00059691A4D2040294008435861C0460395A0
:101CB00090250020ED050294C04666461969009CF7
:101CC000090A215401326969D2B2940031402600D8
:101CD0003E4031436961039E596901303140029EA3
:101CE000C0B234400C4301995C618842E4D90823B6
:101CF000AB62DB18AB6105B0F0BDC0460004004824
:101D000000005555FFFFAAAAFFFC000003FF0000DA
:101D1000F0B585B00193284B284C1D6800902C43EA
:101D20001C6027485C691F2943D880252943090284
:101D3000E4B2214359610221996199621968214CE9
:101D40000840902118608020C90588624869950084
:101D5000C026A44620402C00B60034402043FF2477
:101D600048615869184F2540384005435D61C046B9
:101D7000002002960394C0461D69009C2D0A25543C
:101D800064464D6901322540D2B2029C960034402F
:101D900025434D61039C5D6926403D400130019C17
:101DA0002E43C0B25E61A042E5D980238B6105B0AD
:101DB000F0BDE4B20902BCE700040048000055553C
:101DC000FFFFAAAAFFFC000003FF0000002302009F
:101DD0000002002A04D1002B01D080231843704751
:101DE000DB43511EDBB20A40F3E70023800080B2E0
:101DF000C046C04601339BB29842F9D17047FFFFFD
:101E00009022D205F0B553691B4C86002340C024B4
:101E1000A400344023435361184B194D5C69000AF8
:101E20002C40FF252E4034435C611E68154C000297
:101E300026431E605E69144F2E40304358610220D5
:101E400098619862186810263840186008209062DF
:101E500096621868090204431C60586928400143CF
:101E60005961C04601219962C046996119680F40C5
:101E70001F609661F0BDC046FFFC000000040048F2
:101E800003FF000000005555FFFFAAAA9022D205CB
:101E90005369194930B50B40C021840089002140A5
:101EA0000B435361154B164D5969000A2940FF2514
:101EB0002C40214359611C681249000221431960DA
:101EC000596908240D40022128435861996199629B
:101ED00019680D48802501401960102194619162B4
:101EE0009562C046C046C0461869E0409561C0B2E0
:101EF0009462916130BDC046FFFC000000040048C0
:101F000003FF000000005555FFFFAAAA1D4B30B586
:101F1000984202D880231B0218439025ED056B6977
:101F2000194C82002340C024A400144023436B6159
:101F3000164B174D5C69000A2C40FF252A401443BC
:101F40005C611C68134A000214431C605C6909024E
:101F50002C40204358610220986198621C680E480A
:101F600004401C601C6822431A605A692A401143CD
:101F70005961C04601229A62C0469A611A680240BD
:101F80001A6030BDFF1F0000FFFC00000004004885
:101F900003FF000000005555FFFFAAAA1A4B30B5F9
:101FA000984202D880231B0218439021C9054B692F
:101FB000164A84001340C0229200224013434B6112
:101FC000134B144D5A69000A2A40FF252C40224326
:101FD0005A611C68104A000222431A605A6915406F
:101FE0000222284358619A619A621A680B4802409B
:101FF0001A6080228A62C046C046C046C046186940
:10200000000AC0B28A6130BDFF1F0000FFFC000063
:102010000004004803FF000000005555FFFFAAAA76
:1020200070B504000D000D48AA21FFF76FFF552180
:102030000B48FFF76BFFA0210848FFF767FF290057
:102040002000FFF763FF2000FFF7A8FF0500C04650
:102050002000FFF7A3FFA842F5D170BD5515000081
:10206000AA1A000070B504000D000D48AA21FFF760
:102070004DFF55210B48FFF749FFA0210848FFF706
:1020800045FF29002000FFF741FF2000FFF786FFF2
:102090000500C0462000FFF781FFA842F5D170BDC2
:1020A00055150000AA0A00009022F0B50124D205BF
:1020B00013688500A3431360D368204EA343D36005
:1020C00053691F4C09022340C024A4002C40234321
:1020D00053611C4B5C693440FF2635402C435C61E6
:1020E0001D68194C25431D605F69050A37402D02A4
:1020F0003D435D6102259D619D621F68134D00B2E5
:102100002F401F60202797621F683C431C605C695A
:1021100034402143596108219161002801DA4918AE
:102120009162C046C0460821916249189161103100
:1021300091611A6815401D60F0BDC04603FF0000A4
:10214000FFFC00000004004800005555FFFFAAAA4C
:10215000F7B51C4B07001D781B4B01911C882021F3
:1021600026002036B6B23000FFF79EFFAA2117489E
:10217000FFF7CCFE2000103080B21021FFF794FF53
:102180002D0155211248FFF7C1FEEDB2202130008C
:10219000FFF78AFF6419A0210C48FFF7B7FEA0B231
:1021A0002900FFF781FF01993800FFF7AFFE3800E3
:1021B000FFF7F4FE0400C0463800FFF7EFFEA04230
:1021C000F5D1F7BD88040020360400205515000025
:1021D000AA0A000070B50400B0200E0000020A2117
:1021E000FFF762FFC0200A210002FFF75DFFAA216E
:1021F0001248FFF78BFE55211148FFF787FEA021FB
:102200000E48FFF783FEB0200E4B00021D78290018
:10221000FFF74AFFC02029000002FFF745FF310009
:102220002000FFF773FE2000FFF7B8FE0500C04650
:102230002000FFF7B3FEA842F5D170BD5515000090
:10224000AA0A000088040020F8B505000E00194B0A
:1022500002211C88A71CBFB23800FFF725FFAA2166
:102260001548FFF753FE601C80B20121FFF71CFFE9
:1022700055211248FFF74AFE02213800FFF714FFEC
:10228000A0210D48FFF742FE0D4B19786418A0B24B
:10229000FFF70AFF31002800FFF738FE2800FFF79C
:1022A0007DFE0400C0462800FFF778FEA042F5D16D
:1022B000F8BDC0463604002055150000AA0A0000EB
:1022C0008804002070B59024E40563691A4AFF264B
:1022D0001340C022850092002A4013436361174BCC
:1022E000174A596935401140294359611968154AFF
:1022F0000A431A605969020A0E40120232435A61B7
:1023000002229A619A621A680F4900B20A401A6062
:102310000822A261002801DA9218A262C046C046D3
:10232000C046C046186990230822DB059A62000A5D
:102330009218C0B29A6170BDFFFC00000004004812
:1023400003FF000000005555FFFFAAAA70B5040066
:102350000D001048AA21FFF7A7FE55210E48FFF7F0
:10236000A3FEA0210B48FFF79FFE29002000FFF7E6
:102370009BFEA020094B00021978FFF795FE200074
:10238000FFF7A0FF0500C0462000FFF79BFFA84213
:10239000F5D170BDAAFA000055F5000088040020B0
:1023A00070B504000D001048AA21FFF77DFE5521ED
:1023B0000E48FFF779FEA0210B48FFF775FE2900B4
:1023C0002000FFF771FE802000210002FFF76CFE65
:1023D0002000FFF777FF0500C0462000FFF772FFDF
:1023E000A842F5D170BDC04655D50000AAAA00008C
:1023F0009022D205536970B5194C86002340C02441
:10240000A400344023435361164B174C5D69000A06
:102410002540FF24264035435D611E68134D0002B0
:102420002E431E605E690902264030435861022037
:102430009861986218680E4E30401860186805431D
:102440001D6058692040014359610121106808430B
:102450001060916291611A6816401E6070BDC0469E
:10246000FFFC00000004004803FF00000000555579
:10247000FFFFAAAA9022D205536970B51B4C8600B3
:102480002340C024A400344023435361184B194D0A
:102490005C69000A2C40FF252E4034435C611E68B5
:1024A000154C000226431E605E6909022E4030432F
:1024B00058610220986198621E68104806401E60AC
:1024C0001E6834431C605C69254029435961012121
:1024D00014680C431460916214688C431460D468CF
:1024E0002143D1601A681040186070BDFFFC0000E5
:1024F0000004004803FF000000005555FFFFAAAA92
:1025000070B505000E00134B00211C882000FFF75A
:10251000CBFDAA211048FFF7ADFF55210F48FFF76B
:10252000A9FFA0210C48FFF7A5FF0D4B19786418EF
:10253000A0B2FFF7B9FD31002800FFF79BFF28008C
:10254000FFF7C0FE0400C0462800FFF7BBFEA04214
:10255000F5D170BD3604002055550000AA2A0000B0
:102560008804002070B504000D000D48AA21FFF773
:1025700081FF55210B48FFF77DFFA0210848FFF799
:1025800079FF29002000FFF775FF2000FFF79AFE72
:1025900005002000FFF796FEA842F6D170BDC046A8
:1025A00055550000AA2A0000F0B5284B85B01E78CA
:1025B000274B01901B78029100930392254B112821
:1025C00040D00022902000251A70C0051C782A00F7
:1025D0002B00012184460198202805D1009D1D4132
:1025E0000D4231D00C430D00029820280ED1002B53
:1025F00001D1174FBB54604607690F4206D01448FB
:10260000875C080098400743114887540398013EAF
:10261000F6B2002804D0002E02D102200D0004439F
:102620000133DBB2082B05D10132094BD2B29B5CDE
:1026300000930023002ECED1002D01D0054B1C703D
:1026400005B0F0BD0122BDE78C43CCE7D9040020E2
:10265000B904002094040020F0B5134B134D1978F1
:102660000023112800D102230027114E3A00B4465E
:102670003C0001262B702B7820280CD163461B5D73
:102680003700134101323340D2B25B00082A02D135
:1026900000220134E4B20139C9B20029ECD1002F83
:1026A00000D02B70F0BDC046D90400209404002057
:1026B000B904002000230B4A012113709022D20597
:1026C000106888431060D0680143D1608021064AB9
:1026D00011701900054A1370054A99540133202BD3
:1026E000FBD1704794040020DA040020D9040020B4
:1026F000B904002010B52B4B1B78082B4ED013D8F3
:10270000294C032B39D006D8012B28D0022B2AD0F4
:10271000254BEE223AE0062B3AD03DD8042BF7D1D8
:1027200001222021112021E00F2B28D008D81E4C97
:102730000D2B1FD000220E2BEAD12021102015E0F6
:10274000802B06D0184CFF2B06D0102BE0D1002296
:102750001FE0FFF7AFFF10BDF0232370FBE7202041
:10276000FFF77AFF04E0012200212020FFF71CFF81
:102770008223F2E700221100F7E70122DDE70022C1
:1027800020211120FFF710FF8222074B1A70E2E789
:10279000012220210800E9E71020E1E71120FFF7DE
:1027A0005BFFF1E7B8040020DA040020BC235B499A
:1027B000DB038A6AF0B513438B628B6A584A594D22
:1027C00013408B62E0234A691B0313434B61902340
:1027D0004022DB051868802690431860D868F6040C
:1027E0000243DA601A685048802702401A6080224B
:1027F000D86852000243DA601A684C48FF0202406F
:102800001A608022D868D2000243DA601A68484809
:1028100002401A608022D868D20102430120DA60A7
:10282000444A146884431460D4680443D4601C6828
:102830002C401C608024DD6864032C43DC601C6831
:102840003D4D2C401C608024DD68E4052C43DC6099
:102850001C683A4D2C401C60DC68394D3443DC6008
:102860001C68384E2C401C608024DD6864012C43B9
:10287000DC6004241568A5431560D5682543D56040
:102880001D6885431D60DD688543DD604869384308
:102890004861106830401060D5682B480543D5600A
:1028A000C0254F69ED023D434D6115682C4314600E
:1028B0000224A02594621C68ED022C431C6017685A
:1028C000224C27431760224C1F6827401F6017685F
:1028D000204C27401760DF681C4C3D438027DD609B
:1028E000D368FF021C43D4604B69144D3B434B61DA
:1028F000136833401360D3680343D36013681E40EA
:1029000016608026D368F6041843134BD0601A680B
:102910002A401A60DA683243DA60F0BD00100240E3
:10292000FFFFA1FFFFFFEFFFFFFEFFFFFFFBFFFF2A
:10293000FFBFFFFF00040048FFFFFFBFFFFFFFFBDB
:10294000FFEFFFFFFFFFAAAA0000555550550000FA
:10295000FFFFFAFFAFAAFFFF00080048F7B5802786
:102960000D0001924C7A000203B2A6B20093FF045C
:102970002B7AB34202D26C720020FEBD00986B68C5
:102980002043195D80B2019B98476B681A5D0B4B21
:10299000824206D01A683A431A60802292019A61F4
:1029A000E6E71A68064901340A401A60DA68013617
:1029B0003A43DA60E4B2B6B2DAE7C046000800484B
:1029C000FFFFFFFBF7B50D001600FF27000203B263
:1029D0004C7A01932A7AE3B2A24202D26B720020AF
:1029E000FEBD20006A683840D15C019B0134184369
:1029F00080B2B047A4B2EDE7022907D10F4B104ACD
:102A0000984218D0904209D1180007E0032906D156
:102A10000A4B0B490B4A98420BD108007047042916
:102A2000FCD1064B064A984205D006499042F4D0A4
:102A3000054A8842E6D11000F0E7C046380400207D
:102A40004C040020600400207404002070B50600CF
:102A50000D0005243000013CFFF734FCE4B22900EE
:102A60003000FFF721FB6D08002CF3D170BDFFFF94
:102A700070B50400A0200D0000020221FFF7E6FF60
:102A8000AA211048FFF742FA55210F48FFF73EFAF6
:102A9000A0210C48FFF73AFAA0200C4B000219784D
:102AA000FFF7D4FF29002000FFF730FA2000FFF7DE
:102AB00075FA0500C0462000FFF770FAA842F5D16C
:102AC00070BDC04655150000AA0A00008804002009
:102AD00070B50400C0200D0000020521FFF7B6FF0D
:102AE000AA210D48FFF7E0FA55210C48FFF7DCFA60
:102AF000A0210948FFF7D8FA29002000FFF7D4FAEF
:102B00002000FFF7DFFB0500C0462000FFF7DAFBDF
:102B1000A842F5D170BDC04655550000AAAA0000D4
:102B2000F7B501230225294F01923A780091054318
:102B300093400421A020264E2D049BB229433268E5
:102B4000C00100F0B5FD040001283DD13B7809200B
:102B50009C4005437830A3B232682900FF3000F072
:102B6000A7FD040001282FD13B7832689C40290042
:102B7000A3B2002000F09CFD0400012824D1009B9A
:102B8000180AFFF723F93B7832689C402900A3B26A
:102B900000F08EFD0400012816D16B461878FFF76F
:102BA00015F922003B7829009A4093B2326800F070
:102BB0007FFD0198FFF70AF93B7832689C402900B5
:102BC000A3B200F075FD0400E0B2FEBD00070020D6
:102BD000FC060020F7B501230225274F00903A7824
:102BE0000191054393400421C020244E2D049BB243
:102BF00029433268800100F05BFD0400012838D1D0
:102C000009231D433B78C0209C403268A3B22900B1
:102C1000400000F04DFD040001282AD13B783268C5
:102C20009C402900A3B2002000F042FD04000128CE
:102C30001FD1019B180AFFF7C9F83B7832689C4006
:102C40002900A3B200F034FD0400012811D16B4625
:102C50001879FFF7BBF822003B789A4093B2009AAC
:102C600014430922E1B209041143326800F020FD47
:102C70000400A0B2FEBDC04600070020FC060020F4
:102C80009022CE4B12031968F0B50A431A608022D5
:102C900089B0920219681142FCD0012259680A4396
:102CA0005A608022596852020A435A608022596849
:102CB00052030A435A608022196852040A431A6078
:102CC0008022920419681142FCD011210224BC4ACE
:102CD000BC4D11605A680E398A4322435A608022E3
:102CE000196B0A431A638022D96912040A43DA6114
:102CF000B54BEB81BC231B689847B44B6B82B44B3C
:102D00002B8262B6B34BB44A1A60B44A1A60A0224E
:102D100012015C609A600293029BDB68002BFBD17E
:102D2000029BAF4C1C60FFF741FDF022AD4B0794B6
:102D30001A70029B079AAC4E1A6032782023110059
:102D40009943D2291BD1A949A948C978C37802243B
:102D5000FF2904D1FF3B1C00631E9C41E4B2A54B3C
:102D6000DB78FF2B00D00324A34BDB78FF2B00D0B4
:102D70000424A24BA24F1C703860D22A49D0337869
:102D8000F22B05D10022023B33709D4B1B68DA7099
:102D90003578D02D00D043E1994E3068C378802B30
:102DA00000D03DE1954B1978FFF726FE00233060F7
:102DB000C570068804004372C07AF5B21038132833
:102DC00000D92BE1FDF7D8FB53008B00F5002A0159
:102DD0002A012A012A012A012A012A012A012A019B
:102DE0002A012A012A012A01280035004B0050003F
:102DF0002100FFF701FE01230135EDB2A542F7D313
:102E0000002B00D0386080223B68DA70D02333700A
:102E1000B5E700230125F1E7E17B0F2900D913E293
:102E200009013143237AA278C9B26068FEF70EFF28
:102E30000BE03C23E17B0A009A4300D004E2237AB2
:102E4000A27829436068FEF763FF60726C4B1B68D1
:102E500019889A7A52181A80D822DA70E0E0237A18
:102E6000A278E17B2943E0E7E17B3F23E3E7E37BD3
:102E70001E2B0BD1C020B6092233F1B200029D43B4
:102E8000FFF712F9237AA2788021EBE71C2B0FD1F0
:102E9000A0208121C001FFF707F98020F609F1B2D7
:102EA0000002FFF701F9A0200021C001FFF7FCF8A4
:102EB0008023E27B5B421F2A05D01D43EDB2237ABB
:102EC000A2782900B1E77022A02021889543090942
:102ED0001D43C9B2C001EDB2FFF7E6F8EFE7E37BAF
:102EE000FE2BB3D17609F1B24648FFF70FF86368BD
:102EF000454A0393A378FF260193237AC0270493BE
:102F0000424BBF0019680A431F211A605A690D40DD
:102F10002D0232402A435A6102229A619A621A684B
:102F20003B490A401A6090220821D2059161491854
:102F3000916270319162019950698D0035498C46DA
:102F400008402900394008435061596932483540EA
:102F500001400D435D61C046002106900596C046C4
:102F60001869039D000A685490250198ED05013009
:102F7000C0B201906869019D0131AE0065462840EC
:102F800035003D4028439025ED0568615869069D50
:102F9000C9B22840059D2E40064304985E618842D0
:102FA000DDD280239361783B936208339361617231
:102FB0004CE7237AA278602154E7C0460010024013
:102FC00000200240006000403CA5FFFF41080008CF
:102FD0008508000800300040CCCC000055550000AA
:102FE000AAAA0000DA040020980400204C04002063
:102FF000380400206004002074040020960400209F
:103000008C040020FF3F00000000555500040048DC
:10301000FFFFAAAAFFFC000003FF0000C323E37028
:10302000DB4B1D78F02D00D016E3DA4E3468E378E0
:10303000982B00D010E3D84B20001978FFF7DCFC68
:1030400000233060C370E37AE5702678112B00D13D
:1030500065E2122B00D1F5E2102B00D0FAE2E37BFF
:10306000002B06D130008038C0B2CC4A2100FFF7D7
:1030700075FCE37B012B06D130008038C0B2C84A12
:103080002100FFF79FFCE37B032B06D13000803843
:10309000C0B2C44A2100FFF795FCE37B042B06D1A4
:1030A00030008038C0B2C04A2100FFF757FCE37BF4
:1030B0000A2B06D130008038C0B2BC4A2100FFF78D
:1030C00081FCE37BFD2B15D13F20238830409B09F9
:1030D00003936B4680261B7B06430593677ABBB23E
:1030E000019333021BB20693237A019A934200D3D1
:1030F000ACE06772E37B1E2B11D13F20304080266D
:10310000238806439B09DBB20493657A33021BB222
:10311000AFB20593237ABB4200D3E4E06572E37B50
:103120000C2B17D11F20304080260643C020258855
:10313000A5216D09EDB2C001FEF7B6FF29009C483C
:10314000FEF7B2FF677A35023D43237ABB4200D3D4
:1031500044E16772E37B1C2B3BD1A02023888121B3
:10316000DB09DBB2C0010393FEF79EFF80200399C9
:103170000002FEF799FFA0205421C001FEF794FF42
:10318000677AAA21BBB28B480193FEF78DFF5521C8
:103190008948FEF789FF20218648FEF785FF8023B6
:1031A00033431B021BB20593237A019A934200D347
:1031B00031E18020902100026772FEF775FF8020C8
:1031C00000210002FEF770FF8020F0210002FEF7D0
:1031D0006BFFE37B1F2B30D1A0202188C0010909A0
:1031E000C9B2FEF761FFAA217248657AFEF75CFF5B
:1031F00055217148FEF758FF6E482021FEF754FF15
:10320000702380209E434042304340B20302AFB25D
:103210000393237ABB4200D34AE18020902100022D
:103220006572FEF741FF802000210002FEF73CFF9F
:103230008020F0210002FEF737FFF4232288E3709C
:10324000A37A9B18238007E2C423E8E600215B48A9
:10325000FEF72AFFAA215A48FFF7CAF85521594814
:10326000FFF7C6F8A0215648FFF7C2F86B46187B57
:10327000554B0599C01880B2FEF716FF069D63688E
:103280003D43ADB2D95D2800FFF7B2F8C046280033
:10329000FFF718F804902800FFF714F8049B834206
:1032A000F4D163680499DA5D484B8A4212D1019ADD
:1032B0004749013292B201921A6801370A401A60F6
:1032C0008022D968D2040A43DA6080229201FFB2D8
:1032D0009A6209E780221968D2040A431A608022A0
:1032E00092019A6100E7C02001210002FEF7DCFE96
:1032F000AA213848FEF7D8FEC02000210002FEF7C0
:10330000D3FE55213448FEF7CFFEC0200121000234
:10331000FEF7CAFEA0212F48FEF7C6FEC020049982
:103320000002FEF7C1FE059B2B439BB2019363682D
:103330000198595DFEF7B8FEC0460198FEF7C2FF3E
:1033400003900198FEF7BEFF039B8342F4D16368AC
:1033500003995A5D1D4B8A4210D11A681C490135E8
:103360000A401A608022D968D2040A43DA608022B7
:1033700001379201EDB2BFB29A62CBE680221968A2
:10338000D2040A431A60802292019A61C2E6C046C2
:10339000980400208C040020960400206525000875
:1033A000D12A000801250008A12300084D230008A8
:1033B000FFFF0000AA8A00005585000069FD00009B
:1033C00055550000AA2A000069FDFFFF00080048CB
:1033D000FFFFFFFB55950000AAAA0000AA21A548FF
:1033E000FEF762FE5521A448FEF75EFEA021A1482B
:1033F000FEF75AFE63682800D95DFEF755FEC04609
:103400002800FEF75FFF01902800FEF75BFF019B9D
:103410008342F4D199E6A0205421C001FEF744FE76
:10342000059DA0213D43ADB22800FEF73DFE636837
:103430002800D95DFEF738FEC0462800FEF742FF9F
:1034400004902800FEF73EFF049B8342F4D163689A
:10345000049ADB5D894D934212D1019B884A013366
:103460009BB201932B68013713402B608023EA68DD
:10347000DB041343EB6080239B01FFB2AB6293E656
:10348000A0208121C001FEF70FFE802003990002D9
:10349000FEF70AFEA0205421C001FEF705FE80239E
:1034A0002A68DB0413432B6080239B01AB617BE61E
:1034B000039EA0212E43B6B23000FEF7F5FD6368EF
:1034C0003000595DFEF7F0FDC0463000FEF7FAFE11
:1034D00001903000FEF7F6FE019B8342F4D1636851
:1034E00001995A5D654B8A4210D11A6864490135C9
:1034F0000A4080211A60DA68C9040A43DA6080222F
:1035000001379201EDB2BFB29A6282E680211A6859
:10351000C9040A431A60802292019A6179E6E37B2A
:10352000002B04D1574A21003000FFF74BFAE37B10
:10353000012B04D1544A21003000FFF743FAE37B0A
:10354000022B04D1514A21003000FFF73BFAE37B04
:10355000042B04D14E4A21003000FFF733FAE37BFD
:103560000A2B04D14B4A21003000FFF72BFAE37BF2
:103570000B2B04D1484A21003000FFF723FAE37BEC
:10358000FE2B00D059E6218844484909C9B2FEF70C
:10359000BDFCAA214248657AFEF732FC552141481C
:1035A000FEF72EFC3E482021FEF72AFC1F2030406B
:1035B0000302AFB20393237ABB420DD2657290210E
:1035C0000020FEF71DFC00210800FEF719FCF02189
:1035D0000020FEF715FC30E6039EA0212E433000AC
:1035E000FEF70EFC63683000595DFEF709FCC0462B
:1035F0003000FEF74BFC01903000FEF747FC019BCA
:103600008342F4D1636801995A5D1C4B8A4210D100
:103610001A681B4901350A4080211A60DA68C9041A
:103620000A43DA60802201379201EDB2BFB29A629A
:10363000C1E780211A68C9040A431A6080229201F6
:103640009A61B8E730006030174A2100C0B2FFF736
:10365000B9F9F2E5C323E370144B1B78F02B01D1C9
:10366000FFF767FB832B01D0FFF763FBFFF742F8FF
:10367000FFF75FFB55D50000AAAA0000000800482C
:10368000FFFFFFFB65200008712A0008492200089F
:1036900021200008D521000851210008FF3F00002B
:1036A000AA0A000055050000A9200008DA0400203D
:1036B000F0B5474680B4061C081C000C102801D544
:1036C000162700E004270007000F8046FF20014076
:1036D0005468251C1D439C43F60313850AD5C04638
:1036E000C046C046C046C046C046C046948013830C
:1036F000958002E0012000F081F801390AD4381CDD
:1037000000F07CF8C046948013839580C046C04684
:103710007600E2E7381C013800F070F894801383DB
:103720009580042000F06AF8108A184001D0FF202C
:1037300061E0C046C046C046C046C046C046948010
:103740009580108A184055D001200226B04552D0ED
:103750000921168A1E40FCD1012000F04FF8948008
:10376000C0469580C04603E0C046C046C046C0463D
:10377000948095807600108A1840EFF30080400016
:10378000C00F0643381C023800F038F8948095804A
:10379000022000F033F80139EAD513859480012026
:1037A00000F02CF813839580301C8021022399406F
:1037B0000E401BD1002341085E4149085E41490883
:1037C0005E4149085E4149085E4149085E41490839
:1037D0005E4149085E4149085E41760808D34008C9
:1037E000FF21084048400002013004E00E2002E0C2
:1037F000092000E0002080BCB846F0BD0138FDD1B2
:103800007047C04603685A0003D45B005B08C018C9
:103810007047802212061343F9E7C046F0B55746B9
:103820004E46DE464546E0B5814683B092460029C5
:1038300025D04B1E9B46002701935B46FB18DC0FEF
:10384000E4184B466410E5005E193000FFF7DAFF1C
:10385000019B8046A3420BD0280008304844FFF764
:10386000D1FFD04506D80138504509D2671CE4E79E
:10387000504505D9A74202D0631E9B46DDE70026CE
:10388000300003B03CBC90469946A246AB46F0BD22
:10389000012809D0022805D0002801D00020704757
:1038A0000248FCE70248FAE70248F8E7853F0008CB
:1038B0009D3F0008913F000830B5234B83B00500C1
:1038C0008C1E002B26D001A9200000E000BF00289C
:1038D0001CD001992200FFF7A1FF041E16D0FFF7AC
:1038E00091FF6368A864012B2AD0201D002B23DBE5
:1038F000FFF788FF0023E8642B650368002B0FDBCC
:10390000FFF780FF2861002003B030BD00230920AD
:103910002B61F9E70D480E49091AC9100191D9E741
:103920001801000FFFF7B4FF2861431E98410823D8
:10393000404298430930E7E70123E8642B65DCE760
:10394000002305202B61DFE700000000804800080D
:1039500050490008036810B50400DA0705D4483060
:103960009B070ED500F06CFC23685A070ED51A078A
:1039700013D5DB0604D42000D130FF3000F06CFCFE
:1039800010BD00F059FC23685A07F0D42000D03055
:1039900000F05AFC23681A07EBD420005130FF30A6
:1039A00000F056FC2368E4E70368002B00D01B18E6
:1039B00018007047092070477047C04670B5040072
:1039C0000D0008E02B6C2A006361210001202369AF
:1039D0009847082807D1296C2000FFF76DFF0028C1
:1039E000F0D000F083FE0728FBD10020296CFFF700
:1039F000E3FF281D00F00AFCF0B5CE46474680B52F
:103A0000C3682E4C9846A54483690600140004310F
:103A1000402205A8994600F071FE002304AD0493EE
:103A200023E0F0222B6C5200736129007CA800F087
:103A300065FE7CAA31003369200098478A9B070005
:103A40006B6403934B4600950193320033002100D1
:103A50000120C04700281FD1F0227CA95200280075
:103A600000F04CFE0024082F1FD1296C3000FFF716
:103A700023FF611E8C41070009340028D1D0AB6BB5
:103A800010216B644B4621430193009533003200B3
:103A90000120C047002800D009273800F5239B00EB
:103AA0009D440CBC90469946F0BD072FF4D12000F0
:103AB000296CFFF781FF05A800F0A8FB2CFCFFFF95
:103AC000406C704770B5CB6BFAB00B6404000E000D
:103AD0004022043103A800F011FE01235B4202934F
:103AE00006E002AA210023699847050008280AD1A8
:103AF000129B200019000193FFF7DEFE0028F0D092
:103B000009207AB070BD02A8FFF724FF062DF7D177
:103B100031002000FFF752FF10B58261DA6BC160FF
:103B20001A6419000022FFF767FF10BD436970B5E2
:103B30000B64C36804000D00002B15D10A00236933
:103B4000010002209847072807D0082803D1290040
:103B50002000FFF733FF00F0C9FD0020296CFFF7BC
:103B60002BFF281D00F052FB0122FFF745FF00F05C
:103B7000BDFDC046C36810B5002B05D0CB6B00223D
:103B80000B64FFF739FF10BDFFF79CFFFBE7C04652
:103B90007047C046836810B5002B02D00100012099
:103BA000984710BD012906D0002906D0033902200C
:103BB000012900D970470120FCE7002B08D10F2A0A
:103BC00006D8920082185268009B00201A60F1E724
:103BD0000220EFE700B585B003AB0A000093002197
:103BE0000023FFF7DFFF039805B000BD012906D0D1
:103BF000002906D003390220012900D9704701208D
:103C0000FCE7002B08D10F2A06D8009B92001B6806
:103C1000821853600020F1E70220EFE700B585B07D
:103C200003AB039200930A0000230021FFF7DEFF9D
:103C300005B000BD70B51A4CD36BA54413640600E3
:103C40000D0019A8111D402200F058FD01235B4210
:103C5000189314E00C2118A802AAFFF7DFFF29002F
:103C600018A8B047002812D1069B18AA02A908304C
:103C700001939847040005280AD0092807D0289BFB
:103C800002A819000193FFF717FE0028E2D00924CB
:103C900018A8FFF75FFE200090239B009D4470BD95
:103CA000C0FDFFFFF0B5DE4657464E464546E0B53F
:103CB000160003220D0011008BB01F000193EB6C66
:103CC00001401C1D009107A91B688B460894002F1A
:103CD0006BD01A0C1B045946079302230B72FD3359
:103CE00013409B004A72E418009B022B00D1AC6B7E
:103CF0002B6DDB0747D40023059308330340029361
:103D00002768002F00D112E1019B022B49D0638864
:103D1000278898460434012340469A469843AB6C62
:103D20000F21994681443000FFF754FF002181455F
:103D300006D839005346994349448842894149424B
:103D400043465A0002231340012217403B43012BF4
:103D50003AD0002B30D0022B1BD12368009A5F0091
:103D60007F08002A67D1002906D0029A002A00D1D4
:103D70007CE0002F00D1A9E0002B00DA04340137E9
:103D8000BF00E419BCE75946300000F00BFB0028E7
:103D900010D009200BB03CBC90469946A246AB46D9
:103DA000F0BD636808349846B5E71B0207935B468D
:103DB0001A8199E70820EDE7009B002B02D000292B
:103DC00000D08DE004349BE7009B002B1AD1002922
:103DD00016D02368DF0F63689A1CDAD02A005832A5
:103DE0000692013300D1BDE0201DFFF7DDFD06ABDB
:103DF00001003A00280000E000BF002800D082E067
:103E000008347DE70D2130002F6AFFF7E3FE87427B
:103E1000F6D1AB6A9C42F3D12000FFF7F3FC0F21EF
:103E200002003000FFF7FAFE30002A000021FFF701
:103E3000F5FE0720AEE72B6A0D2130009846FFF70C
:103E4000C9FE804501D0236896E7AB6A9C42FAD14F
:103E50000023EB6204332B63231DAF626B63236883
:103E6000002B00DA86E00123059388E7002F2DD090
:103E700058239C46AC4463460393231D9946002374
:103E8000984606AB220004933B004C464746B24698
:103E900098462E00914603E004342F00454542D059
:103EA000039B20000693FFF77FFD049B0100002287
:103EB00030007D1C00E000BF0028EDD04346B8462E
:103EC00035004C4656461F009845BCD10D213000A8
:103ED000FFF780FE069B28626B62AC62062059E702
:103EE0002000FFF78FFC04340700AC63280000E0DB
:103EF00000BF002800D14CE730003A000F21FFF747
:103F00008DFE072046E707000D213000FFF762FE17
:103F10002862022F2BD1069BEB622B002C336B62A5
:103F2000AC62062036E735004C465646CEE7594689
:103F3000300000F037FA002800D02AE7059B002B5C
:103F400000D137E70F213000FFF744FE0E210200B9
:103F50003000FFF763FE3000094A0F21FFF75EFED5
:103F6000072017E70D213000FFF734FE2862069B7B
:103F70006B62D5E738000130800020184DE7C0465D
:103F80000000000010B50023FFF78CFE10BDC046F6
:103F900010B50123FFF786FE10BDC04610B5022301
:103FA000FFF780FE10BDC046F0B5CE46474680B54F
:103FB0000500C3B014001E00012955D000294BD0C4
:103FC000032922D0042949D1002B47D1102A45D8F2
:103FD000102203681A4200D0F1E020AF380000F050
:103FE0003DF900230120A96B02009A40144203D03E
:103FF0000E689A00BE5004310133042BF4D138000E
:10400000A96300F029F9002029E0032B26D114042C
:10401000230C160C9846F318102B1FD8082203689F
:104020001A4200D098E020AF380000F013F9424661
:10403000AB6BF6001C00002A08D0D400F21A1C1941
:10404000BA181968D15004339C42FAD1AC633800D5
:1040500000F0FEF8002002E0002B24D0022043B044
:104060000CBC90469946F0BD130C14049846240CE1
:10407000012E2ED0052EF1D11B19202BEED8424651
:104080000F2A70D9A146002C7ED1AA6B4346AA63A1
:104090000F2B00D89AE04B46002BDBD0684600F08F
:1040A000D3F80020DBE700231004A96B000C0136D5
:1040B00032009A40104204D00F689A00AA18576044
:1040C00004310133102BF3D10020A304C7D4A9631A
:1040D000C5E71B19102BC1D843460F2BBED82B6840
:1040E0001E4206D00322280093432B60483000F084
:1040F000A5F820AF380000F0A1F8AA6B002C24D05E
:104100004346DB00FF180023994664000023A40007
:10411000D158F95004339C42FAD14B4612196F46DC
:10412000002B0FD04046102800D210204B46D9005B
:1041300000231038C0003818D458C45004339942B2
:10414000FAD15218012EA1D120AF04323800AA634F
:1041500000F072F8002082E7934303605130FF3093
:1041600000F078F85FE7102B3BD9102252429146BD
:1041700099442B68194208D0022228008B4313432C
:104180002B60483000F05EF82B6804221A4221D1DF
:1041900043460F2B03D820AF380000F053F86F468A
:1041A000380000F053F810244346AA6BE41A002CA0
:1041B000B8DD434620AFDB006400FF18A6E7934359
:1041C0000360D130FF3000F049F806E720A800F086
:1041D00037F860E7280093432B60D03000F036F8C2
:1041E000D6E72B680B4207D0022228008B431343EB
:1041F0002B60483000F026F820AF380000F022F89D
:10420000A146AA6B002C00D07AE73FE7011C3431AD
:1042100038C9043B9C461D60A646011C20313CC9A0
:1042200090469946A246AB46011C0831FCC941683C
:104230000068E54600BDC0467047C0467047C046AE
:104240007047C0467047C0467047C0467047C0467A
:104250007047C0467047C0467047C0467047C0466A
:1042600001B401A801B585B0FFB408A841464A468B
:1042700053465C4665463EC001A83EC80F98009074
:1042800000230CB401A9FFF71DFC109B12B01847C6
:1042900001B401A801B585B0FFB408A841464A465B
:1042A00053465C4665463EC001A83EC80F98009044
:1042B00000230CB401A9FFF739FC109B12B018477A
:1042C00001B401A801B585B0FFB408A841464A462B
:1042D00053465C4665463EC001A83EC80F98009014
:1042E00000230CB401A9FFF745FC109B12B018473E
:1042F00001B401A801B585B0FFB408A841464A46FB
:1043000053465C4665463EC001A83EC80F980090E3
:1043100000230CB401ABFFF7FFFB109B12B0184752
:1043200001B401A801B585B0FFB408A841464A46CA
:1043300053465C4665463EC001A83EC80F980090B3
:1043400000230CB401AAFFF775FC109B12B01847AC
:10435000027A0300002A0BD1427A002A0FD0013AD8
:1043600042724268111D416003211268017202E02D
:10437000013A02720268100E12021A607047B020F1
:10438000FCE7C04600B585B003AB00930C220023C8
:104390000021FFF707FC039805B000BD10B5FFF73B
:1043A000F1FF10BDF0B557464E464546DE460023A8
:1043B000E0B587B003930F339846083B99468023B6
:1043C0001B0306000F009A463800FFF7C1FF0400E8
:1043D000B02800D1C3E003062AD503004246934328
:1043E000DBB2802B00D171E0902B3DD0A02B00D10F
:1043F00085E0B02B50D0C02B00D196E003004A4698
:104400009343DBB2D02B0AD15346024001321A4308
:10441000052301213000FFF7C7FD0028D4D009246F
:10442000200007B03CBC90469946A246AB46F0BD82
:10443000FF23820013401D1D05AB9B4600930D22F8
:10444000002300213000FFF7ADFB630620D4059B5D
:104450009C46654405955B460D2200930021002390
:104460003000FFF7C3FBAFE7833B03400D2BD6D0F3
:1044700005AD02400095002300213000FFF792FBBC
:10448000009500230D2200213000FFF7AFFB9BE7D2
:10449000059B5D1B0595DEE7B12874D0B22800D1DD
:1044A000CFE0B32800D184E0FC230340B42BB6D086
:1044B0004A465346024001321A430121012330008B
:1044C000FFF772FD002800D17EE7A8E7040238005C
:1044D000FFF73EFF802520432D02A8429FD0040114
:1044E0000005020C002300213000FFF75DFD0028CD
:1044F00095D12C4200D167E70123039364E7FF23A2
:104500004A461B011900824311410A001A40030761
:1045100002D58023DB011A43002300213000FFF77E
:1045200043FD002800D14FE779E7C6284CD0C728C3
:104530005ED003004A469343DBB2C02B6DD0C8283F
:1045400072D0C92800D06AE73800FFF701FFF023D6
:1045500002031B03134042460240013257E7039B0C
:104560000024002B00D05BE705AD00950E22002152
:104570003000FFF717FB009500230F2200213000C9
:10458000FFF734FB4CE73800FFF7E2FE002800D1CC
:1045900045E7030042469343DBB2002B00D03EE7E1
:1045A000020000213000FFF7FFFC002800D10BE7DC
:1045B00035E73800FFF7CCFEF02302031B0313405E
:1045C00042460240013277E73800FFF7C1FEF02390
:1045D00002031B0313404246024001321A430323E5
:1045E00003213000FFF7E0FC002800D1ECE616E7DD
:1045F0003800FFF7ADFE021E00D110E70300414670
:104600008B43DBB2002B00D009E704213000FFF719
:10461000CBFC002800D1D7E601E74346A0221C408E
:10462000013412032243DAE73800FFF791FE4346D4
:1046300002009A43D2B210321840120301300243F2
:10464000E6E605AB00939B460D22002300213000D7
:10465000FFF7A8FA3800FFF77BFE030618D57F2581
:10466000B03C059B2840A0409C4660440590380023
:104670000734FFF76DFE0306F3D481217F23890001
:1046800003408C46A340059A62449B180593E2E6DA
:104690000224F2E7030000B5DB6C85B05A6808001D
:1046A000120201921A0001A908324A6003220A721A
:1046B000DB794B72FFF776FE05B000BD10B5FFF752
:1046C0006DFE806C10BDC04610B5FFF767FEC26C72
:1046D000D3799B000833D01810BDC04610B500F048
:1046E00005F8C04610B5FFF7F9FFC04610B5062023
:1046F00000F076F8012000F0A5F8C046F0B50F2ACA
:1047000037D90D0005430C000300AD0735D1150066
:10471000103D2D092E013618103627681F60676876
:104720005F60A7689F60E7681034DF601033B342B2
:10473000F3D10F2401352D01491914404519032CDB
:104740001DD90023CE58EE500433E61A032EF9D8B3
:104750000323043CA4080134A4001A402D190919AC
:10476000002A05D00023CC5CEC5401339342FAD1EB
:10477000F0BD0500002AF5D1FAE70500F2E72200B6
:10478000F8E7C04670B505000C001F2922D8B723F2
:104790009B00C358002B0ED08A009B181A68002A71
:1047A00009D0012A10D0511C10D00021200019601E
:1047B0009047002070BD280000F030F82200010072
:1047C000280000F017F8F5E70020F3E71623036050
:1047D0000120EFE71623036001204042EAE7C046CC
:1047E00010B5034B01001868FFF7CCFF10BDC046A1
:1047F00000000020002370B5074C050008001100E0
:10480000236000F017F8431C00D070BD2368002B14
:10481000FBD02B60F9E7C0460407002010B500F07C
:1048200001F810BD58220120014B40421A60704728
:104830000407002058220120014B40421A607047B3
:1048400004070020FEE7C046F8B5C046F8B5C046EC
:1048500074B20181B0AB308000000000800A018199
:10486000B0B0ABF0000000003F020181B0AB30807F
:104870000000000080060181B0B0ABF00000000035
:1048800030EEFF7FB0B0B0807CEFFF7F0100000012
:1048900028F0FF7FB0A90280BCF0FF7FB0B0A880F5
:1048A00008F1FF7F0100000014F1FF7FB0B0AA8083
:1048B00048F1FF7F9CFFFF7F08F2FF7F01000000AF
:1048C00004F2FF7FAA3F398050F2FF7FB0B0A8808A
:1048D0005CF2FF7FB0B0AA809CF2FF7FB0B0A880EE
:1048E000B0F2FF7F01000000ACF2FF7FB0B0A88003
:1048F000B4F2FF7F010000003CF3FF7FAA0FB280FB
:10490000A4F3FF7F58FFFF7F7CF6FF7FB0B0A88045
:1049100098F6FF7F54FFFF7FF4F8FF7F010000004F
:1049200064FAFF7F0084048074FAFF7FB0B0A8802F
:1049300074FAFF7F40FFFF7F5CFDFF7F00840480EF
:104940007CFDFF7FB0B0A88094FDFF7F01000000D8
:10495000080000200000000000000000F402002019
:104960005C030020C40300200000000000000000E1
:104970000000000000000000000000000000000037
:104980000000000000000000000000000000000027
:104990000000000000000000000000000000000017
:1049A0000000000000000000000000000000000007
:1049B00000000000000000000000000000000000F7
:1049C00000000000000000000000000000000000E7
:1049D00000000000000000000000000000000000D7
:1049E00000000000000000000000000000000000C7
:1049F00000000000000000000000000000000000B7
:104A000001000000000000000E33CDAB34126DE653
:104A1000ECDE05000B0000000000000000000000BC
:104A20000000000000000000000000000000000086
:104A30000000000000000000000000000000000076
:104A40000000000000000000000000000000000066
:104A50000000000000000000000000000000000056
:0400000508000805E2
:00000001FF
